BL51 BANKED LINKER/LOCATER V5.00                                                        05/05/2011  10:38:39  PAGE 1


BL51 BANKED LINKER/LOCATER V5.00, INVOKED BY:
C:\KEIL中文版\KEIL\C51\BIN\BL51.EXE software.obj TO tem RAMSIZE (256)


MEMORY MODEL: SMALL


INPUT MODULES INCLUDED:
  software.obj (SOFTWARE)
  C:\KEIL中文版\KEIL\C51\LIB\C51S.LIB (?C_STARTUP)
  C:\KEIL中文版\KEIL\C51\LIB\C51S.LIB (?C_INIT)


LINK MAP OF MODULE:  tem (SOFTWARE)


            TYPE    BASE      LENGTH    RELOCATION   SEGMENT NAME
            -----------------------------------------------------

            * * * * * * *   D A T A   M E M O R Y   * * * * * * *
            REG     0000H     0008H     ABSOLUTE     "REG BANK 0"
            DATA    0008H     0002H     UNIT         _DATA_GROUP_
                    000AH     0016H                  *** GAP ***
            BIT     0020H.0   0001H.0   UNIT         ?BI?SOFTWARE
            BIT     0021H.0   0000H.1   UNIT         _BIT_GROUP_
                    0021H.1   0000H.7                *** GAP ***
            DATA    0022H     002CH     UNIT         ?DT?SOFTWARE
            IDATA   004EH     0001H     UNIT         ?STACK

            * * * * * * *   C O D E   M E M O R Y   * * * * * * *
            CODE    0000H     0003H     ABSOLUTE     
                    0003H     0008H                  *** GAP ***
            CODE    000BH     0003H     ABSOLUTE     
            CODE    000EH     000CH     UNIT         ?PR?LCD_CLR?SOFTWARE
                    001AH     0001H                  *** GAP ***
            CODE    001BH     0003H     ABSOLUTE     
            CODE    001EH     0127H     UNIT         ?CO?SOFTWARE
            CODE    0145H     0105H     UNIT         ?PR?ECODECHANGE?SOFTWARE
            CODE    024AH     00AAH     UNIT         ?PR?DISP_TEMPERATURE?SOFTWARE
            CODE    02F4H     0093H     UNIT         ?PR?ECODE?SOFTWARE
            CODE    0387H     008CH     UNIT         ?C_C51STARTUP
            CODE    0413H     0078H     UNIT         ?PR?KEYSCAN?SOFTWARE
            CODE    048BH     006EH     UNIT         ?PR?MAIN?SOFTWARE
            CODE    04F9H     005EH     UNIT         ?PR?SET_TEMP_ALARM?SOFTWARE
            CODE    0557H     0055H     UNIT         ?PR?_DISP_ROMCODE?SOFTWARE
            CODE    05ACH     0050H     UNIT         ?PR?READ_TEMPERATURE?SOFTWARE
            CODE    05FCH     004FH     UNIT         ?PR?LCD_INIT?SOFTWARE
            CODE    064BH     004EH     UNIT         ?PR?_DISP_TEMP_ALARM?SOFTWARE
            CODE    0699H     004DH     UNIT         ?PR?TEMP_COMPARE?SOFTWARE
            CODE    06E6H     003FH     UNIT         ?PR?NATURAL_MENU?SOFTWARE
            CODE    0725H     003BH     UNIT         ?PR?LCD_START?SOFTWARE
            CODE    0760H     0035H     UNIT         ?PR?CRC8?SOFTWARE
            CODE    0795H     0035H     UNIT         ?C_INITSEG
            CODE    07CAH     002CH     UNIT         ?PR?ERROR_MENU?SOFTWARE
            CODE    07F6H     002CH     UNIT         ?PR?ERROR_MENU1?SOFTWARE
            CODE    0822H     002CH     UNIT         ?PR?RIGHT_MENU?SOFTWARE
            CODE    084EH     002CH     UNIT         ?PR?_SHOUT?SOFTWARE
            CODE    087AH     002BH     UNIT         ?PR?KEYDOWN?SOFTWARE
BL51 BANKED LINKER/LOCATER V5.00                                                      05/05/2011  10:38:39  PAGE 2


            CODE    08A5H     0027H     UNIT         ?PR?ROMCODE_MENU?SOFTWARE
            CODE    08CCH     0025H     UNIT         ?PR?_LCD_WCMD?SOFTWARE
            CODE    08F1H     0025H     UNIT         ?PR?FLASH?SOFTWARE
            CODE    0916H     0024H     UNIT         ?PR?_KEY_SET?SOFTWARE
            CODE    093AH     0023H     UNIT         ?PR?INIT_DS18B20?SOFTWARE
            CODE    095DH     0021H     UNIT         ?PR?TIME1?SOFTWARE
            CODE    097EH     0020H     UNIT         ?PR?_DELAYMS?SOFTWARE
            CODE    099EH     0020H     UNIT         ?PR?READONECHAR?SOFTWARE
            CODE    09BEH     0020H     UNIT         ?PR?CODEDISPLAY?SOFTWARE
            CODE    09DEH     0020H     UNIT         ?PR?TEST?SOFTWARE
            CODE    09FEH     001FH     UNIT         ?PR?_WRITEONECHAR?SOFTWARE
            CODE    0A1DH     001FH     UNIT         ?PR?WRITE_TEMPERATURE_ALARM?SOFTWARE
            CODE    0A3CH     001FH     UNIT         ?PR?_SET_TEMPALARM_FLASH?SOFTWARE
            CODE    0A5BH     001EH     UNIT         ?PR?WRITETAB?SOFTWARE
            CODE    0A79H     001EH     UNIT         ?PR?_WRITE_BYTE?SOFTWARE
            CODE    0A97H     001DH     UNIT         ?PR?_LCD_WDAT?SOFTWARE
            CODE    0AB4H     001DH     UNIT         ?PR?TIME0?SOFTWARE
            CODE    0AD1H     001AH     UNIT         ?PR?DELAYS?SOFTWARE
            CODE    0AEBH     0018H     UNIT         ?PR?READ_ROMCORD?SOFTWARE
            CODE    0B03H     0018H     UNIT         ?PR?BEEP?SOFTWARE
            CODE    0B1BH     0017H     UNIT         ?PR?_SPK?SOFTWARE
            CODE    0B32H     0016H     UNIT         ?PR?READ24C02?SOFTWARE
            CODE    0B48H     0015H     UNIT         ?PR?SHIN?SOFTWARE
            CODE    0B5DH     0014H     UNIT         ?PR?LCD_BUSY?SOFTWARE
            CODE    0B71H     0013H     UNIT         ?PR?_READ_RANDOM?SOFTWARE
            CODE    0B84H     0011H     UNIT         ?PR?START?SOFTWARE
            CODE    0B95H     0010H     UNIT         ?PR?_DELAY?SOFTWARE
            CODE    0BA5H     0010H     UNIT         ?PR?_LCD_POS?SOFTWARE
            CODE    0BB5H     000FH     UNIT         ?PR?STOP?SOFTWARE
            CODE    0BC4H     000FH     UNIT         ?PR?READ_CURRENT?SOFTWARE



OVERLAY MAP OF MODULE:   tem (SOFTWARE)


SEGMENT                                         BIT_GROUP          DATA_GROUP 
  +--> CALLED SEGMENT                        START    LENGTH     START    LENGTH
--------------------------------------------------------------------------------
?C_C51STARTUP                                -----    -----      -----    -----
  +--> ?PR?MAIN?SOFTWARE
  +--> ?C_INITSEG

?PR?MAIN?SOFTWARE                            -----    -----      -----    -----
  +--> ?PR?READ24C02?SOFTWARE
  +--> ?PR?LCD_START?SOFTWARE
  +--> ?PR?ECODE?SOFTWARE
  +--> ?PR?INIT_DS18B20?SOFTWARE
  +--> ?PR?ERROR_MENU?SOFTWARE
  +--> ?PR?BEEP?SOFTWARE
  +--> ?PR?ROMCODE_MENU?SOFTWARE
  +--> ?PR?_DELAY?SOFTWARE
  +--> ?PR?NATURAL_MENU?SOFTWARE
  +--> ?PR?READ_TEMPERATURE?SOFTWARE
  +--> ?PR?DISP_TEMPERATURE?SOFTWARE
  +--> ?PR?TEMP_COMPARE?SOFTWARE
  +--> ?PR?SET_TEMP_ALARM?SOFTWARE
BL51 BANKED LINKER/LOCATER V5.00                                                      05/05/2011  10:38:39  PAGE 3



?PR?READ24C02?SOFTWARE                       -----    -----      -----    -----
  +--> ?PR?_READ_RANDOM?SOFTWARE

?PR?_READ_RANDOM?SOFTWARE                    -----    -----      -----    -----
  +--> ?PR?START?SOFTWARE
  +--> ?PR?_SHOUT?SOFTWARE
  +--> ?PR?READ_CURRENT?SOFTWARE

?PR?_SHOUT?SOFTWARE                          0021H.0  0000H.1    -----    -----

?PR?READ_CURRENT?SOFTWARE                    -----    -----      -----    -----
  +--> ?PR?START?SOFTWARE
  +--> ?PR?_SHOUT?SOFTWARE
  +--> ?PR?SHIN?SOFTWARE
  +--> ?PR?STOP?SOFTWARE

?PR?LCD_START?SOFTWARE                       -----    -----      -----    -----
  +--> ?PR?LCD_INIT?SOFTWARE
  +--> ?PR?_LCD_POS?SOFTWARE
  +--> ?PR?LCD_CLR?SOFTWARE
  +--> ?CO?SOFTWARE
  +--> ?PR?_LCD_WDAT?SOFTWARE
  +--> ?PR?_DELAYMS?SOFTWARE
  +--> ?PR?FLASH?SOFTWARE

?PR?LCD_INIT?SOFTWARE                        -----    -----      -----    -----
  +--> ?PR?_DELAYMS?SOFTWARE
  +--> ?PR?_LCD_WCMD?SOFTWARE
  +--> ?PR?WRITETAB?SOFTWARE

?PR?_LCD_WCMD?SOFTWARE                       -----    -----      -----    -----
  +--> ?PR?_DELAYMS?SOFTWARE
  +--> ?PR?LCD_BUSY?SOFTWARE

?PR?LCD_BUSY?SOFTWARE                        0021H.0  0000H.1    -----    -----

?PR?WRITETAB?SOFTWARE                        -----    -----      -----    -----
  +--> ?PR?_LCD_WCMD?SOFTWARE
  +--> ?CO?SOFTWARE
  +--> ?PR?_LCD_WDAT?SOFTWARE

?PR?_LCD_WDAT?SOFTWARE                       -----    -----      -----    -----
  +--> ?PR?LCD_BUSY?SOFTWARE

?PR?_LCD_POS?SOFTWARE                        -----    -----      -----    -----
  +--> ?PR?_DELAYMS?SOFTWARE
  +--> ?PR?_LCD_WCMD?SOFTWARE

?PR?LCD_CLR?SOFTWARE                         -----    -----      -----    -----
  +--> ?PR?_LCD_WCMD?SOFTWARE
  +--> ?PR?_DELAYMS?SOFTWARE

?PR?FLASH?SOFTWARE                           -----    -----      -----    -----
  +--> ?PR?_DELAYMS?SOFTWARE
  +--> ?PR?_LCD_WCMD?SOFTWARE

BL51 BANKED LINKER/LOCATER V5.00                                                      05/05/2011  10:38:39  PAGE 4


?PR?ECODE?SOFTWARE                           -----    -----      -----    -----
  +--> ?PR?_LCD_POS?SOFTWARE
  +--> ?PR?LCD_CLR?SOFTWARE
  +--> ?CO?SOFTWARE
  +--> ?PR?_LCD_WDAT?SOFTWARE
  +--> ?PR?_DELAYMS?SOFTWARE
  +--> ?PR?FLASH?SOFTWARE
  +--> ?PR?KEYDOWN?SOFTWARE
  +--> ?PR?ERROR_MENU1?SOFTWARE
  +--> ?PR?DELAYS?SOFTWARE
  +--> ?PR?RIGHT_MENU?SOFTWARE

?PR?KEYDOWN?SOFTWARE                         -----    -----      -----    -----
  +--> ?PR?KEYSCAN?SOFTWARE
  +--> ?PR?BEEP?SOFTWARE
  +--> ?PR?DELAYS?SOFTWARE
  +--> ?PR?ECODECHANGE?SOFTWARE

?PR?KEYSCAN?SOFTWARE                         -----    -----      -----    -----
  +--> ?PR?_DELAYMS?SOFTWARE

?PR?BEEP?SOFTWARE                            -----    -----      -----    -----
  +--> ?PR?_DELAY?SOFTWARE

?PR?ECODECHANGE?SOFTWARE                     -----    -----      0008H    0002H
  +--> ?PR?LCD_CLR?SOFTWARE
  +--> ?PR?_LCD_POS?SOFTWARE
  +--> ?CO?SOFTWARE
  +--> ?PR?_LCD_WDAT?SOFTWARE
  +--> ?PR?_DELAYMS?SOFTWARE
  +--> ?PR?DELAYS?SOFTWARE
  +--> ?PR?ERROR_MENU1?SOFTWARE
  +--> ?PR?_WRITE_BYTE?SOFTWARE

?PR?ERROR_MENU1?SOFTWARE                     -----    -----      -----    -----
  +--> ?PR?LCD_INIT?SOFTWARE
  +--> ?PR?_LCD_POS?SOFTWARE
  +--> ?CO?SOFTWARE
  +--> ?PR?_LCD_WDAT?SOFTWARE

?PR?_WRITE_BYTE?SOFTWARE                     -----    -----      -----    -----
  +--> ?PR?START?SOFTWARE
  +--> ?PR?_SHOUT?SOFTWARE
  +--> ?PR?STOP?SOFTWARE
  +--> ?PR?_DELAYMS?SOFTWARE

?PR?RIGHT_MENU?SOFTWARE                      -----    -----      -----    -----
  +--> ?PR?LCD_INIT?SOFTWARE
  +--> ?PR?_LCD_POS?SOFTWARE
  +--> ?CO?SOFTWARE
  +--> ?PR?_LCD_WDAT?SOFTWARE

?PR?INIT_DS18B20?SOFTWARE                    -----    -----      -----    -----
  +--> ?PR?_DELAY?SOFTWARE

?PR?ERROR_MENU?SOFTWARE                      -----    -----      -----    -----
  +--> ?PR?LCD_INIT?SOFTWARE
BL51 BANKED LINKER/LOCATER V5.00                                                      05/05/2011  10:38:39  PAGE 5


  +--> ?PR?_LCD_POS?SOFTWARE
  +--> ?CO?SOFTWARE
  +--> ?PR?_LCD_WDAT?SOFTWARE

?PR?ROMCODE_MENU?SOFTWARE                    -----    -----      -----    -----
  +--> ?PR?LCD_INIT?SOFTWARE
  +--> ?PR?_LCD_POS?SOFTWARE
  +--> ?CO?SOFTWARE
  +--> ?PR?_LCD_WDAT?SOFTWARE
  +--> ?PR?READ_ROMCORD?SOFTWARE
  +--> ?PR?CRC8?SOFTWARE
  +--> ?PR?_DISP_ROMCODE?SOFTWARE

?PR?READ_ROMCORD?SOFTWARE                    -----    -----      -----    -----
  +--> ?PR?INIT_DS18B20?SOFTWARE
  +--> ?PR?_WRITEONECHAR?SOFTWARE
  +--> ?PR?READONECHAR?SOFTWARE

?PR?_WRITEONECHAR?SOFTWARE                   -----    -----      -----    -----
  +--> ?PR?INIT_DS18B20?SOFTWARE
  +--> ?PR?_DELAY?SOFTWARE

?PR?READONECHAR?SOFTWARE                     -----    -----      -----    -----
  +--> ?PR?_DELAY?SOFTWARE

?PR?_DISP_ROMCODE?SOFTWARE                   -----    -----      -----    -----
  +--> ?PR?_LCD_POS?SOFTWARE
  +--> ?PR?_LCD_WDAT?SOFTWARE

?PR?NATURAL_MENU?SOFTWARE                    -----    -----      -----    -----
  +--> ?PR?LCD_INIT?SOFTWARE
  +--> ?PR?_LCD_POS?SOFTWARE
  +--> ?CO?SOFTWARE
  +--> ?PR?_LCD_WDAT?SOFTWARE
  +--> ?PR?READ_TEMPERATURE?SOFTWARE
  +--> ?PR?_DISP_TEMP_ALARM?SOFTWARE
  +--> ?PR?DISP_TEMPERATURE?SOFTWARE

?PR?READ_TEMPERATURE?SOFTWARE                -----    -----      -----    -----
  +--> ?PR?_WRITEONECHAR?SOFTWARE
  +--> ?PR?INIT_DS18B20?SOFTWARE
  +--> ?PR?READONECHAR?SOFTWARE

?PR?_DISP_TEMP_ALARM?SOFTWARE                -----    -----      -----    -----
  +--> ?PR?_LCD_POS?SOFTWARE
  +--> ?PR?_LCD_WDAT?SOFTWARE

?PR?DISP_TEMPERATURE?SOFTWARE                -----    -----      -----    -----
  +--> ?PR?_LCD_POS?SOFTWARE
  +--> ?PR?_LCD_WDAT?SOFTWARE

?PR?TEMP_COMPARE?SOFTWARE                    -----    -----      -----    -----
  +--> ?PR?_SPK?SOFTWARE
  +--> ?PR?BEEP?SOFTWARE
  +--> ?PR?_LCD_POS?SOFTWARE
  +--> ?PR?_LCD_WDAT?SOFTWARE

BL51 BANKED LINKER/LOCATER V5.00                                                      05/05/2011  10:38:39  PAGE 6


?PR?_SPK?SOFTWARE                            -----    -----      -----    -----
  +--> ?PR?_LCD_POS?SOFTWARE
  +--> ?PR?_LCD_WDAT?SOFTWARE

?PR?SET_TEMP_ALARM?SOFTWARE                  -----    -----      -----    -----
  +--> ?PR?BEEP?SOFTWARE
  +--> ?PR?_KEY_SET?SOFTWARE
  +--> ?PR?_SET_TEMPALARM_FLASH?SOFTWARE
  +--> ?PR?WRITE_TEMPERATURE_ALARM?SOFTWARE

?PR?_KEY_SET?SOFTWARE                        -----    -----      -----    -----
  +--> ?PR?BEEP?SOFTWARE

?PR?_SET_TEMPALARM_FLASH?SOFTWARE            -----    -----      -----    -----
  +--> ?PR?_DISP_TEMP_ALARM?SOFTWARE
  +--> ?PR?_LCD_POS?SOFTWARE
  +--> ?PR?_LCD_WDAT?SOFTWARE

?PR?WRITE_TEMPERATURE_ALARM?SOFTWARE         -----    -----      -----    -----
  +--> ?PR?_WRITEONECHAR?SOFTWARE



SYMBOL TABLE OF MODULE:  tem (SOFTWARE)

  VALUE           TYPE          NAME
  ----------------------------------

  -------         MODULE        SOFTWARE
  C:0000H         SYMBOL        _ICE_DUMMY_
  B:0090H.7       PUBLIC        K4
  C:0557H         PUBLIC        _Disp_RomCode
  D:0080H         PUBLIC        P0
  D:0090H         PUBLIC        P1
  D:00A0H         PUBLIC        P2
  C:02F4H         PUBLIC        ecode
  D:00B0H         PUBLIC        P3
  B:00B0H.4       PUBLIC        T0
  B:00D0H.6       PUBLIC        AC
  C:07CAH         PUBLIC        Error_Menu
  C:0699H         PUBLIC        temp_compare
  B:00B0H.5       PUBLIC        T1
  C:087AH         PUBLIC        keydown
  C:0AD4H         PUBLIC        delays
  B:00A8H.7       PUBLIC        EA
  C:0BC4H         PUBLIC        read_current
  C:00D9H         PUBLIC        cdis10
  C:00E5H         PUBLIC        cdis11
  C:0A3CH         PUBLIC        _Set_tempalarm_Flash
  C:024AH         PUBLIC        Disp_Temperature
  C:00F1H         PUBLIC        cdis12
  C:0102H         PUBLIC        cdis13
  C:0113H         PUBLIC        cdis15
  C:0062H         PUBLIC        cdis33
  C:0124H         PUBLIC        cdis16
  C:0074H         PUBLIC        cdis44
  C:0760H         PUBLIC        CRC8
BL51 BANKED LINKER/LOCATER V5.00                                                      05/05/2011  10:38:39  PAGE 7


  C:08F1H         PUBLIC        flash
  C:0A03H         PUBLIC        _WriteOneChar
  B:00A0H.3       PUBLIC        DQ
  C:084EH         PUBLIC        _shout
  B:00B0H.7       PUBLIC        RD
  D:0022H         PUBLIC        Temp
  B:00A8H.4       PUBLIC        ES
  C:09BEH         PUBLIC        codedisplay
  C:0AEBH         PUBLIC        Read_RomCord
  B:0098H.0       PUBLIC        RI
  B:0020H.0       PUBLIC        flag
  B:00B0H.2       PUBLIC        INT0
  B:00D0H.7       PUBLIC        CY
  C:093AH         PUBLIC        Init_DS18B20
  B:00A0H.4       PUBLIC        BEEP
  B:0098H.1       PUBLIC        TI
  B:00B0H.3       PUBLIC        INT1
  C:0B03H         PUBLIC        beep
  C:08D5H         PUBLIC        _lcd_wcmd
  C:099EH         PUBLIC        ReadOneChar
  B:00B8H.4       PUBLIC        PS
  C:0A79H         PUBLIC        _write_byte
  C:08A5H         PUBLIC        RomCode_Menu
  B:00D0H.2       PUBLIC        OV
  C:048BH         PUBLIC        main
  C:0A9AH         PUBLIC        _lcd_wdat
  D:0023H         PUBLIC        temp_alarm
  B:0020H.1       PUBLIC        compare_th
  B:00B0H.6       PUBLIC        WR
  D:0025H         PUBLIC        count
  D:0026H         PUBLIC        display1
  D:0029H         PUBLIC        RomCode
  B:0020H.2       PUBLIC        compare_tl
  C:0B1BH         PUBLIC        _spk
  C:0B84H         PUBLIC        start
  C:0B48H         PUBLIC        shin
  D:0031H         PUBLIC        ecode1
  D:003BH         PUBLIC        ecode2
  D:0041H         PUBLIC        temp_data
  D:0089H         PUBLIC        TMOD
  C:07F6H         PUBLIC        Error_Menu1
  D:0043H         PUBLIC        crc
  B:0088H.1       PUBLIC        IE0
  B:0088H.3       PUBLIC        IE1
  C:0AB4H         PUBLIC        Time0
  C:09DEH         PUBLIC        test
  C:095DH         PUBLIC        Time1
  C:0725H         PUBLIC        lcd_start
  B:00A0H.2       PUBLIC        LCD_EN
  C:0BB5H         PUBLIC        stop
  C:0BAEH         PUBLIC        _lcd_pos
  B:00A8H.1       PUBLIC        ET0
  D:0044H         PUBLIC        key
  D:0045H         PUBLIC        temp_comp
  B:00A8H.3       PUBLIC        ET1
  B:0088H.5       PUBLIC        TF0
  C:0B32H         PUBLIC        read24c02
BL51 BANKED LINKER/LOCATER V5.00                                                      05/05/2011  10:38:39  PAGE 8


  C:05FCH         PUBLIC        lcd_init
  B:0088H.7       PUBLIC        TF1
  B:0098H.2       PUBLIC        RB8
  D:008CH         PUBLIC        TH0
  B:0020H.3       PUBLIC        flag1
  B:00A8H.0       PUBLIC        EX0
  B:0088H.0       PUBLIC        IT0
  B:0098H.3       PUBLIC        TB8
  B:00A8H.2       PUBLIC        EX1
  B:0088H.2       PUBLIC        IT1
  B:00D0H.0       PUBLIC        P
  B:0098H.7       PUBLIC        SM0
  D:008AH         PUBLIC        TL0
  C:0B9BH         PUBLIC        _Delay
  C:0135H         PUBLIC        mytab1
  B:0098H.6       PUBLIC        SM1
  C:013DH         PUBLIC        mytab2
  B:0098H.5       PUBLIC        SM2
  C:06E6H         PUBLIC        Natural_Menu
  C:0984H         PUBLIC        _delayms
  B:00B8H.1       PUBLIC        PT0
  B:00B8H.3       PUBLIC        PT1
  B:00D0H.3       PUBLIC        RS0
  C:001EH         PUBLIC        cdis1
  B:0088H.4       PUBLIC        TR0
  B:00D0H.4       PUBLIC        RS1
  C:000EH         PUBLIC        lcd_clr
  C:04F9H         PUBLIC        set_temp_alarm
  C:002FH         PUBLIC        cdis2
  B:0088H.6       PUBLIC        TR1
  C:0916H         PUBLIC        _key_set
  C:0040H         PUBLIC        cdis3
  B:00B0H.5       PUBLIC        SDA
  B:00B8H.0       PUBLIC        PX0
  C:0051H         PUBLIC        cdis4
  B:00A0H.0       PUBLIC        LCD_RS
  B:00B8H.2       PUBLIC        PX1
  C:0B5DH         PUBLIC        lcd_busy
  C:0085H         PUBLIC        cdis5
  B:0020H.4       PUBLIC        presence
  C:064BH         PUBLIC        _Disp_Temp_alarm
  C:0096H         PUBLIC        cdis6
  C:00A7H         PUBLIC        cdis7
  C:00B8H         PUBLIC        cdis8
  B:00A0H.1       PUBLIC        LCD_RW
  D:0046H         PUBLIC        timecount
  C:00C9H         PUBLIC        cdis9
  B:00B0H.4       PUBLIC        SCL
  C:0B71H         PUBLIC        _read_random
  B:0098H.4       PUBLIC        REN
  C:0A5BH         PUBLIC        writetab
  D:0047H         PUBLIC        temp1
  D:0048H         PUBLIC        k
  B:0020H.5       PUBLIC        alarm_on_off
  C:0145H         PUBLIC        ecodechange
  B:00B0H.0       PUBLIC        RXD
  B:00B0H.1       PUBLIC        TXD
BL51 BANKED LINKER/LOCATER V5.00                                                      05/05/2011  10:38:39  PAGE 9


  C:0413H         PUBLIC        keyscan
  C:05ACH         PUBLIC        Read_Temperature
  C:0A1DH         PUBLIC        Write_Temperature_alarm
  B:0020H.6       PUBLIC        temp_th
  B:00D0H.5       PUBLIC        F0
  C:0822H         PUBLIC        RIGHT_Menu
  B:0020H.7       PUBLIC        temp_tl
  D:0049H         PUBLIC        display
  B:0090H.4       PUBLIC        K1
  B:0090H.5       PUBLIC        K2
  B:0090H.6       PUBLIC        K3
  -------         PROC          L?0283
  -------         ENDPROC       L?0283
  -------         PROC          _DELAY
  D:0006H         SYMBOL        num
  C:0B9BH         LINE#         78
  C:0B9BH         LINE#         79
  C:0B9BH         LINE#         80
  C:0BA4H         LINE#         81
  -------         ENDPROC       _DELAY
  C:097EH         SYMBOL        L?0273
  C:0980H         SYMBOL        L?0274
  -------         PROC          L?0272
  -------         ENDPROC       L?0272
  C:097EH         SYMBOL        L?0273
  C:0980H         SYMBOL        L?0274
  -------         PROC          _DELAYMS
  D:0006H         SYMBOL        ms
  -------         DO            
  D:0005H         SYMBOL        y
  -------         ENDDO         
  C:0984H         LINE#         89
  C:0984H         LINE#         90
  C:0984H         LINE#         92
  C:098EH         LINE#         93
  C:098EH         LINE#         94
  C:0996H         LINE#         95
  C:0996H         LINE#         96
  C:0997H         LINE#         97
  C:0998H         LINE#         98
  C:0999H         LINE#         99
  C:099AH         LINE#         100
  C:099DH         LINE#         101
  C:099DH         LINE#         102
  -------         ENDPROC       _DELAYMS
  -------         PROC          L?0280
  -------         ENDPROC       L?0280
  -------         PROC          DELAYS
  C:0AD4H         LINE#         108
  C:0AD4H         LINE#         109
  C:0AD4H         LINE#         110
  C:0ADDH         LINE#         111
  C:0AE5H         LINE#         112
  C:0AE8H         LINE#         113
  C:0AEAH         LINE#         114
  -------         ENDPROC       DELAYS
  -------         PROC          TIME1
BL51 BANKED LINKER/LOCATER V5.00                                                      05/05/2011  10:38:39  PAGE 10


  C:095DH         LINE#         118
  C:0961H         LINE#         120
  C:0964H         LINE#         121
  C:0967H         LINE#         122
  C:0969H         LINE#         123
  C:096EH         LINE#         124
  C:096EH         LINE#         125
  C:0971H         LINE#         126
  C:0973H         LINE#         127
  C:0979H         LINE#         128
  C:0979H         LINE#         129
  -------         ENDPROC       TIME1
  -------         PROC          LCD_BUSY
  -------         DO            
  B:0021H.0       SYMBOL        result
  -------         ENDDO         
  C:0B5DH         LINE#         140
  C:0B5DH         LINE#         141
  C:0B5DH         LINE#         143
  C:0B5FH         LINE#         144
  C:0B61H         LINE#         145
  C:0B63H         LINE#         146
  C:0B67H         LINE#         147
  C:0B6CH         LINE#         148
  C:0B6EH         LINE#         149
  C:0B70H         LINE#         150
  -------         ENDPROC       LCD_BUSY
  C:08CEH         SYMBOL        L?0279
  -------         PROC          L?0278
  -------         ENDPROC       L?0278
  C:08CEH         SYMBOL        L?0279
  -------         PROC          _LCD_WCMD
  D:0007H         SYMBOL        cmd
  C:08D5H         LINE#         158
  C:08D5H         LINE#         159
  C:08D5H         LINE#         160
  C:08DAH         LINE#         161
  C:08DCH         LINE#         162
  C:08DEH         LINE#         163
  C:08E0H         LINE#         164
  C:08E1H         LINE#         165
  C:08E2H         LINE#         166
  C:08E4H         LINE#         167
  C:08E8H         LINE#         168
  C:08EAH         LINE#         169
  C:08EEH         LINE#         170
  C:08F0H         LINE#         171
  -------         ENDPROC       _LCD_WCMD
  -------         PROC          L?0275
  -------         ENDPROC       L?0275
  -------         PROC          _LCD_WDAT
  D:0007H         SYMBOL        dat
  C:0A9AH         LINE#         179
  C:0A9AH         LINE#         180
  C:0A9AH         LINE#         181
  C:0A9FH         LINE#         182
  C:0AA1H         LINE#         183
BL51 BANKED LINKER/LOCATER V5.00                                                      05/05/2011  10:38:39  PAGE 11


  C:0AA3H         LINE#         184
  C:0AA5H         LINE#         185
  C:0AA7H         LINE#         186
  C:0AABH         LINE#         187
  C:0AADH         LINE#         188
  C:0AB1H         LINE#         189
  C:0AB3H         LINE#         190
  -------         ENDPROC       _LCD_WDAT
  -------         PROC          WRITETAB
  -------         DO            
  D:0006H         SYMBOL        i
  -------         ENDDO         
  C:0A5BH         LINE#         197
  C:0A5BH         LINE#         198
  C:0A5BH         LINE#         200
  C:0A60H         LINE#         201
  C:0A62H         LINE#         202
  C:0A6CH         LINE#         203
  C:0A6EH         LINE#         204
  C:0A78H         LINE#         205
  -------         ENDPROC       WRITETAB
  -------         PROC          LCD_CLR
  C:000EH         LINE#         213
  C:000EH         LINE#         214
  C:000EH         LINE#         215
  C:0013H         LINE#         216
  -------         ENDPROC       LCD_CLR
  -------         PROC          FLASH
  C:08F1H         LINE#         224
  C:08F1H         LINE#         225
  C:08F1H         LINE#         226
  C:08F8H         LINE#         227
  C:08FDH         LINE#         228
  C:08FDH         LINE#         229
  C:0900H         LINE#         230
  C:0907H         LINE#         231
  C:090CH         LINE#         232
  C:090CH         LINE#         233
  C:090FH         LINE#         234
  -------         ENDPROC       FLASH
  -------         PROC          LCD_INIT
  C:05FCH         LINE#         242
  C:05FCH         LINE#         243
  C:05FCH         LINE#         244
  C:0603H         LINE#         245
  C:0608H         LINE#         246
  C:060DH         LINE#         247
  C:0614H         LINE#         248
  C:0619H         LINE#         249
  C:0620H         LINE#         250
  C:0625H         LINE#         251
  C:0627H         LINE#         253
  C:062AH         LINE#         254
  C:0631H         LINE#         255
  C:0636H         LINE#         256
  C:063CH         LINE#         257
  C:0641H         LINE#         258
BL51 BANKED LINKER/LOCATER V5.00                                                      05/05/2011  10:38:39  PAGE 12


  C:0648H         LINE#         260
  -------         ENDPROC       LCD_INIT
  C:0BA5H         SYMBOL        L?0277
  -------         PROC          L?0276
  -------         ENDPROC       L?0276
  C:0BA5H         SYMBOL        L?0277
  -------         PROC          _LCD_POS
  D:0007H         SYMBOL        pos
  C:0BAEH         LINE#         269
  C:0BAEH         LINE#         270
  C:0BAEH         LINE#         271
  -------         ENDPROC       _LCD_POS
  -------         PROC          INIT_DS18B20
  C:093AH         LINE#         283
  C:093AH         LINE#         284
  C:093AH         LINE#         285
  C:093AH         LINE#         286
  C:093DH         LINE#         288
  C:093FH         LINE#         289
  C:0946H         LINE#         291
  C:0946H         LINE#         292
  C:0949H         LINE#         294
  C:094DH         LINE#         295
  C:0954H         LINE#         296
  C:0956H         LINE#         298
  C:095CH         LINE#         299
  -------         ENDPROC       INIT_DS18B20
  -------         PROC          READONECHAR
  -------         DO            
  D:0005H         SYMBOL        i
  D:0004H         SYMBOL        dat
  -------         ENDDO         
  C:099EH         LINE#         306
  C:099EH         LINE#         307
  C:099EH         LINE#         308
  C:099FH         LINE#         309
  C:09A0H         LINE#         311
  C:09A2H         LINE#         312
  C:09A2H         LINE#         313
  C:09A4H         LINE#         314
  C:09A8H         LINE#         315
  C:09AAH         LINE#         317
  C:09ADH         LINE#         318
  C:09B0H         LINE#         319
  C:09B7H         LINE#         320
  C:09B9H         LINE#         321
  C:09BDH         LINE#         322
  -------         ENDPROC       READONECHAR
  C:09FEH         SYMBOL        L?0282
  -------         PROC          L?0281
  -------         ENDPROC       L?0281
  C:09FEH         SYMBOL        L?0282
  -------         PROC          _WRITEONECHAR
  D:0005H         SYMBOL        dat
  -------         DO            
  D:0003H         SYMBOL        i
  -------         ENDDO         
BL51 BANKED LINKER/LOCATER V5.00                                                      05/05/2011  10:38:39  PAGE 13


  C:0A03H         LINE#         329
  C:0A05H         LINE#         330
  C:0A05H         LINE#         331
  C:0A05H         LINE#         332
  C:0A07H         LINE#         333
  C:0A07H         LINE#         334
  C:0A09H         LINE#         335
  C:0A0DH         LINE#         336
  C:0A14H         LINE#         338
  C:0A16H         LINE#         339
  C:0A1AH         LINE#         340
  C:0A1CH         LINE#         341
  -------         ENDPROC       _WRITEONECHAR
  -------         PROC          WRITE_TEMPERATURE_ALARM
  C:0A1DH         LINE#         348
  C:0A1DH         LINE#         349
  C:0A1DH         LINE#         350
  C:0A1DH         LINE#         352
  C:0A20H         LINE#         353
  C:0A25H         LINE#         354
  C:0A2AH         LINE#         355
  C:0A2FH         LINE#         356
  C:0A34H         LINE#         358
  C:0A34H         LINE#         359
  C:0A37H         LINE#         360
  -------         ENDPROC       WRITE_TEMPERATURE_ALARM
  -------         PROC          READ_ROMCORD
  -------         DO            
  D:0003H         SYMBOL        j
  -------         ENDDO         
  C:0AEBH         LINE#         368
  C:0AEBH         LINE#         369
  C:0AEBH         LINE#         371
  C:0AEEH         LINE#         373
  C:0AF3H         LINE#         374
  C:0AF5H         LINE#         375
  C:0AF5H         LINE#         376
  C:0AFEH         LINE#         377
  C:0B02H         LINE#         378
  -------         ENDPROC       READ_ROMCORD
  -------         PROC          CRC8
  -------         DO            
  D:0005H         SYMBOL        i
  D:0007H         SYMBOL        x
  D:0006H         SYMBOL        crcbuff
  -------         ENDDO         
  C:0760H         LINE#         385
  C:0760H         LINE#         386
  C:0760H         LINE#         389
  C:0763H         LINE#         390
  C:0764H         LINE#         391
  C:0764H         LINE#         392
  C:076AH         LINE#         393
  C:076CH         LINE#         394
  C:076CH         LINE#         395
  C:0772H         LINE#         396
  C:077AH         LINE#         397
BL51 BANKED LINKER/LOCATER V5.00                                                      05/05/2011  10:38:39  PAGE 14


  C:077AH         LINE#         398
  C:077DH         LINE#         399
  C:0783H         LINE#         400
  C:0786H         LINE#         401
  C:0786H         LINE#         402
  C:078AH         LINE#         403
  C:078EH         LINE#         404
  C:0792H         LINE#         405
  C:0794H         LINE#         406
  -------         ENDPROC       CRC8
  -------         PROC          _DISP_ROMCODE
  D:0006H         SYMBOL        H_num
  -------         DO            
  D:0006H         SYMBOL        j
  -------         ENDDO         
  C:0557H         LINE#         413
  C:0559H         LINE#         414
  C:0559H         LINE#         417
  C:055CH         LINE#         418
  C:0561H         LINE#         419
  C:0564H         LINE#         420
  C:0569H         LINE#         422
  C:056BH         LINE#         423
  C:056BH         LINE#         424
  C:0572H         LINE#         426
  C:0579H         LINE#         427
  C:057EH         LINE#         428
  C:0582H         LINE#         429
  C:0588H         LINE#         430
  C:058DH         LINE#         432
  C:0593H         LINE#         433
  C:0598H         LINE#         434
  C:059CH         LINE#         435
  C:05A2H         LINE#         436
  C:05A7H         LINE#         437
  C:05ABH         LINE#         438
  -------         ENDPROC       _DISP_ROMCODE
  -------         PROC          READ_TEMPERATURE
  -------         DO            
  D:0004H         SYMBOL        i
  -------         ENDDO         
  C:05ACH         LINE#         445
  C:05ACH         LINE#         446
  C:05ACH         LINE#         448
  C:05AEH         LINE#         449
  C:05AEH         LINE#         451
  C:05B1H         LINE#         452
  C:05B6H         LINE#         454
  C:05B9H         LINE#         456
  C:05BEH         LINE#         457
  C:05C0H         LINE#         458
  C:05CDH         LINE#         460
  C:05D2H         LINE#         462
  C:05D7H         LINE#         463
  C:05DCH         LINE#         464
  C:05E1H         LINE#         465
  C:05E6H         LINE#         467
BL51 BANKED LINKER/LOCATER V5.00                                                      05/05/2011  10:38:39  PAGE 15


  C:05F9H         LINE#         469
  C:05FBH         LINE#         470
  -------         ENDPROC       READ_TEMPERATURE
  -------         PROC          DISP_TEMPERATURE
  -------         DO            
  D:0007H         SYMBOL        s
  -------         ENDDO         
  C:024AH         LINE#         476
  C:024AH         LINE#         477
  C:024AH         LINE#         478
  C:024CH         LINE#         479
  C:0253H         LINE#         480
  C:0253H         LINE#         481
  C:0259H         LINE#         482
  C:025EH         LINE#         483
  C:0266H         LINE#         484
  C:0269H         LINE#         485
  C:026BH         LINE#         486
  C:026BH         LINE#         488
  C:0271H         LINE#         489
  C:027CH         LINE#         491
  C:028FH         LINE#         492
  C:0297H         LINE#         493
  C:02A0H         LINE#         494
  C:02AAH         LINE#         495
  C:02B6H         LINE#         497
  C:02BBH         LINE#         498
  C:02BBH         LINE#         499
  C:02BEH         LINE#         500
  C:02C3H         LINE#         501
  C:02C6H         LINE#         502
  C:02C6H         LINE#         503
  C:02C9H         LINE#         504
  C:02CCH         LINE#         506
  C:02D1H         LINE#         507
  C:02D6H         LINE#         508
  C:02DBH         LINE#         509
  C:02E0H         LINE#         510
  C:02E5H         LINE#         511
  C:02EAH         LINE#         512
  C:02EFH         LINE#         513
  -------         ENDPROC       DISP_TEMPERATURE
  -------         PROC          BEEP
  -------         DO            
  D:0005H         SYMBOL        y
  -------         ENDDO         
  C:0B03H         LINE#         521
  C:0B03H         LINE#         522
  C:0B03H         LINE#         524
  C:0B05H         LINE#         525
  C:0B05H         LINE#         526
  C:0B0CH         LINE#         527
  C:0B0EH         LINE#         528
  C:0B12H         LINE#         529
  C:0B14H         LINE#         530
  -------         ENDPROC       BEEP
  -------         PROC          ROMCODE_MENU
BL51 BANKED LINKER/LOCATER V5.00                                                      05/05/2011  10:38:39  PAGE 16


  -------         DO            
  D:0006H         SYMBOL        m
  -------         ENDDO         
  C:08A5H         LINE#         538
  C:08A5H         LINE#         539
  C:08A5H         LINE#         541
  C:08A8H         LINE#         543
  C:08ADH         LINE#         544
  C:08AFH         LINE#         545
  C:08BCH         LINE#         547
  C:08BFH         LINE#         548
  C:08C2H         LINE#         549
  C:08C6H         LINE#         550
  C:08C6H         LINE#         551
  C:08CBH         LINE#         552
  C:08CBH         LINE#         553
  -------         ENDPROC       ROMCODE_MENU
  -------         PROC          ERROR_MENU
  -------         DO            
  D:0006H         SYMBOL        m
  -------         ENDDO         
  C:07CAH         LINE#         560
  C:07CAH         LINE#         561
  C:07CAH         LINE#         563
  C:07CDH         LINE#         565
  C:07D2H         LINE#         566
  C:07D4H         LINE#         567
  C:07E1H         LINE#         569
  C:07E6H         LINE#         570
  C:07E8H         LINE#         571
  C:07F5H         LINE#         572
  -------         ENDPROC       ERROR_MENU
  -------         PROC          ERROR_MENU1
  -------         DO            
  D:0006H         SYMBOL        m
  -------         ENDDO         
  C:07F6H         LINE#         578
  C:07F6H         LINE#         579
  C:07F6H         LINE#         581
  C:07F9H         LINE#         583
  C:07FEH         LINE#         584
  C:0800H         LINE#         585
  C:080DH         LINE#         587
  C:0812H         LINE#         588
  C:0814H         LINE#         589
  C:0821H         LINE#         590
  -------         ENDPROC       ERROR_MENU1
  -------         PROC          RIGHT_MENU
  -------         DO            
  D:0006H         SYMBOL        m
  -------         ENDDO         
  C:0822H         LINE#         596
  C:0822H         LINE#         597
  C:0822H         LINE#         599
  C:0825H         LINE#         601
  C:082AH         LINE#         602
  C:082CH         LINE#         603
BL51 BANKED LINKER/LOCATER V5.00                                                      05/05/2011  10:38:39  PAGE 17


  C:0839H         LINE#         605
  C:083EH         LINE#         606
  C:0840H         LINE#         607
  C:084DH         LINE#         608
  -------         ENDPROC       RIGHT_MENU
  -------         PROC          NATURAL_MENU
  -------         DO            
  D:0006H         SYMBOL        m
  -------         ENDDO         
  C:06E6H         LINE#         616
  C:06E6H         LINE#         617
  C:06E6H         LINE#         619
  C:06E9H         LINE#         621
  C:06EEH         LINE#         622
  C:06F0H         LINE#         623
  C:06FDH         LINE#         625
  C:0702H         LINE#         626
  C:0704H         LINE#         627
  C:0711H         LINE#         629
  C:0714H         LINE#         630
  C:071BH         LINE#         631
  C:0722H         LINE#         632
  -------         ENDPROC       NATURAL_MENU
  -------         PROC          START
  C:0B84H         LINE#         643
  C:0B84H         LINE#         645
  C:0B84H         LINE#         646
  C:0B86H         LINE#         647
  C:0B88H         LINE#         648
  C:0B8CH         LINE#         649
  C:0B8EH         LINE#         650
  C:0B92H         LINE#         651
  C:0B94H         LINE#         652
  -------         ENDPROC       START
  -------         PROC          STOP
  C:0BB5H         LINE#         657
  C:0BB5H         LINE#         659
  C:0BB5H         LINE#         660
  C:0BB7H         LINE#         661
  C:0BBBH         LINE#         662
  C:0BBDH         LINE#         663
  C:0BC1H         LINE#         664
  C:0BC3H         LINE#         665
  -------         ENDPROC       STOP
  -------         PROC          SHIN
  -------         DO            
  D:0006H         SYMBOL        i
  D:0007H         SYMBOL        read_data
  -------         ENDDO         
  C:0B48H         LINE#         670
  C:0B48H         LINE#         671
  C:0B48H         LINE#         673
  C:0B4AH         LINE#         674
  C:0B4AH         LINE#         675
  C:0B4CH         LINE#         676
  C:0B50H         LINE#         678
  C:0B56H         LINE#         679
BL51 BANKED LINKER/LOCATER V5.00                                                      05/05/2011  10:38:39  PAGE 18


  C:0B58H         LINE#         680
  C:0B5CH         LINE#         681
  C:0B5CH         LINE#         682
  -------         ENDPROC       SHIN
  -------         PROC          _SHOUT
  D:0007H         SYMBOL        write_data
  -------         DO            
  D:0006H         SYMBOL        i
  B:0021H.0       SYMBOL        ack_bit
  -------         ENDDO         
  C:084EH         LINE#         687
  C:084EH         LINE#         688
  C:084EH         LINE#         691
  C:0850H         LINE#         692
  C:0850H         LINE#         693
  C:0854H         LINE#         694
  C:0855H         LINE#         695
  C:0857H         LINE#         696
  C:085BH         LINE#         697
  C:085DH         LINE#         698
  C:0861H         LINE#         699
  C:0865H         LINE#         700
  C:0867H         LINE#         701
  C:086BH         LINE#         702
  C:086DH         LINE#         703
  C:0871H         LINE#         704
  C:0875H         LINE#         705
  C:0877H         LINE#         706
  C:0879H         LINE#         707
  -------         ENDPROC       _SHOUT
  -------         PROC          _WRITE_BYTE
  D:0004H         SYMBOL        addr
  D:0005H         SYMBOL        write_data
  C:0A79H         LINE#         712
  C:0A7BH         LINE#         713
  C:0A7BH         LINE#         714
  C:0A7EH         LINE#         715
  C:0A83H         LINE#         716
  C:0A88H         LINE#         717
  C:0A8DH         LINE#         718
  C:0A90H         LINE#         719
  -------         ENDPROC       _WRITE_BYTE
  -------         PROC          READ_CURRENT
  -------         DO            
  D:0007H         SYMBOL        read_data
  -------         ENDDO         
  C:0BC4H         LINE#         725
  C:0BC4H         LINE#         726
  C:0BC4H         LINE#         728
  C:0BC7H         LINE#         729
  C:0BCCH         LINE#         730
  C:0BCFH         LINE#         731
  C:0BD2H         LINE#         732
  C:0BD2H         LINE#         733
  -------         ENDPROC       READ_CURRENT
  -------         PROC          _READ_RANDOM
  D:0005H         SYMBOL        random_addr
BL51 BANKED LINKER/LOCATER V5.00                                                      05/05/2011  10:38:39  PAGE 19


  C:0B71H         LINE#         738
  C:0B73H         LINE#         740
  C:0B73H         LINE#         741
  C:0B76H         LINE#         742
  C:0B7BH         LINE#         743
  C:0B80H         LINE#         744
  C:0B83H         LINE#         745
  -------         ENDPROC       _READ_RANDOM
  -------         PROC          CODEDISPLAY
  -------         DO            
  D:0004H         SYMBOL        m
  -------         ENDDO         
  C:09BEH         LINE#         749
  C:09BEH         LINE#         750
  C:09BEH         LINE#         751
  C:09C0H         LINE#         752
  C:09C3H         LINE#         753
  C:09C3H         LINE#         754
  C:09C6H         LINE#         757
  C:09C9H         LINE#         758
  C:09D1H         LINE#         759
  C:09D1H         LINE#         760
  C:09D4H         LINE#         761
  C:09D8H         LINE#         762
  C:09D8H         LINE#         763
  C:09DBH         LINE#         764
  C:09DDH         LINE#         765
  -------         ENDPROC       CODEDISPLAY
  -------         PROC          LCD_START
  -------         DO            
  D:0004H         SYMBOL        m
  -------         ENDDO         
  C:0725H         LINE#         773
  C:0725H         LINE#         774
  C:0725H         LINE#         775
  C:0727H         LINE#         776
  C:072AH         LINE#         777
  C:072AH         LINE#         778
  C:072DH         LINE#         781
  C:0730H         LINE#         782
  C:0738H         LINE#         783
  C:0738H         LINE#         784
  C:073BH         LINE#         785
  C:073FH         LINE#         786
  C:0741H         LINE#         787
  C:0743H         LINE#         788
  C:0748H         LINE#         789
  C:074FH         LINE#         790
  C:074FH         LINE#         791
  C:075BH         LINE#         792
  C:075DH         LINE#         794
  -------         ENDPROC       LCD_START
  -------         PROC          KEYSCAN
  C:0413H         LINE#         800
  C:0413H         LINE#         801
  C:0413H         LINE#         802
  C:0416H         LINE#         803
BL51 BANKED LINKER/LOCATER V5.00                                                      05/05/2011  10:38:39  PAGE 20


  C:0419H         LINE#         804
  C:041CH         LINE#         805
  C:0423H         LINE#         806
  C:0426H         LINE#         807
  C:042BH         LINE#         808
  C:0430H         LINE#         809
  C:0435H         LINE#         810
  C:043AH         LINE#         811
  C:043FH         LINE#         812
  C:0444H         LINE#         813
  C:0449H         LINE#         815
  C:044CH         LINE#         817
  C:044FH         LINE#         818
  C:0452H         LINE#         819
  C:0455H         LINE#         820
  C:0458H         LINE#         821
  C:0462H         LINE#         822
  C:0465H         LINE#         823
  C:0469H         LINE#         824
  C:046EH         LINE#         825
  C:0472H         LINE#         826
  C:0477H         LINE#         827
  C:047BH         LINE#         828
  C:0480H         LINE#         829
  C:0487H         LINE#         831
  C:048AH         LINE#         833
  -------         ENDPROC       KEYSCAN
  -------         PROC          KEYDOWN
  C:087AH         LINE#         838
  C:087AH         LINE#         839
  C:087AH         LINE#         840
  C:087DH         LINE#         841
  C:0883H         LINE#         842
  C:0886H         LINE#         843
  C:0889H         LINE#         845
  C:088EH         LINE#         846
  C:088EH         LINE#         847
  C:088EH         LINE#         848
  C:0891H         LINE#         849
  C:0894H         LINE#         850
  C:0899H         LINE#         851
  C:0899H         LINE#         852
  C:089CH         LINE#         853
  C:089FH         LINE#         854
  C:089FH         LINE#         855
  C:089FH         LINE#         856
  C:08A4H         LINE#         859
  -------         ENDPROC       KEYDOWN
  -------         PROC          ECODE
  -------         DO            
  D:0004H         SYMBOL        m
  -------         ENDDO         
  C:02F4H         LINE#         863
  C:02F4H         LINE#         864
  C:02F4H         LINE#         866
  C:02F6H         LINE#         867
  C:02FAH         LINE#         868
BL51 BANKED LINKER/LOCATER V5.00                                                      05/05/2011  10:38:39  PAGE 21


  C:02FDH         LINE#         869
  C:0304H         LINE#         870
  C:0304H         LINE#         871
  C:0310H         LINE#         872
  C:0312H         LINE#         873
  C:0315H         LINE#         874
  C:0317H         LINE#         875
  C:031BH         LINE#         876
  C:031EH         LINE#         877
  C:0325H         LINE#         878
  C:0325H         LINE#         879
  C:0331H         LINE#         880
  C:0333H         LINE#         881
  C:0336H         LINE#         882
  C:0336H         LINE#         883
  C:0339H         LINE#         884
  C:0340H         LINE#         885
  C:0348H         LINE#         886
  C:034DH         LINE#         887
  C:0356H         LINE#         888
  C:0359H         LINE#         889
  C:0359H         LINE#         890
  C:0369H         LINE#         891
  C:0369H         LINE#         892
  C:036CH         LINE#         893
  C:036FH         LINE#         894
  C:0372H         LINE#         895
  C:0375H         LINE#         896
  C:0375H         LINE#         897
  C:037EH         LINE#         898
  C:0381H         LINE#         899
  C:0384H         LINE#         900
  -------         ENDPROC       ECODE
  -------         PROC          ECODECHANGE
  -------         DO            
  D:0008H         SYMBOL        m
  D:0009H         SYMBOL        k
  -------         ENDDO         
  C:0145H         LINE#         905
  C:0145H         LINE#         906
  C:0145H         LINE#         907
  C:0148H         LINE#         908
  C:014BH         LINE#         909
  C:0150H         LINE#         911
  C:0159H         LINE#         912
  C:0159H         LINE#         913
  C:015CH         LINE#         914
  C:015FH         LINE#         915
  C:0161H         LINE#         916
  C:0164H         LINE#         917
  C:0168H         LINE#         919
  C:0171H         LINE#         920
  C:0171H         LINE#         921
  C:0174H         LINE#         922
  C:0177H         LINE#         923
  C:0179H         LINE#         924
  C:017EH         LINE#         925
BL51 BANKED LINKER/LOCATER V5.00                                                      05/05/2011  10:38:39  PAGE 22


  C:0181H         LINE#         926
  C:0186H         LINE#         927
  C:0189H         LINE#         928
  C:0189H         LINE#         929
  C:018CH         LINE#         930
  C:0193H         LINE#         931
  C:019BH         LINE#         932
  C:01A0H         LINE#         933
  C:01A9H         LINE#         934
  C:01ACH         LINE#         935
  C:01ACH         LINE#         936
  C:01BCH         LINE#         937
  C:01BCH         LINE#         938
  C:01BFH         LINE#         939
  C:01C2H         LINE#         940
  C:01C5H         LINE#         941
  C:01C8H         LINE#         942
  C:01C8H         LINE#         943
  C:01D1H         LINE#         944
  C:01D4H         LINE#         945
  C:01D7H         LINE#         946
  C:01E0H         LINE#         947
  C:01E0H         LINE#         948
  C:01E3H         LINE#         949
  C:01E6H         LINE#         950
  C:01E8H         LINE#         951
  C:01EBH         LINE#         952
  C:01EEH         LINE#         954
  C:01F1H         LINE#         955
  C:01F6H         LINE#         956
  C:01F9H         LINE#         957
  C:0202H         LINE#         958
  C:0202H         LINE#         959
  C:0205H         LINE#         960
  C:0208H         LINE#         961
  C:020AH         LINE#         963
  C:020DH         LINE#         964
  C:020DH         LINE#         965
  C:0210H         LINE#         966
  C:0217H         LINE#         967
  C:021FH         LINE#         968
  C:0224H         LINE#         969
  C:022DH         LINE#         970
  C:022FH         LINE#         971
  C:0231H         LINE#         972
  C:0234H         LINE#         973
  C:0234H         LINE#         974
  C:0240H         LINE#         975
  C:0249H         LINE#         977
  -------         ENDPROC       ECODECHANGE
  -------         PROC          READ24C02
  -------         DO            
  D:0004H         SYMBOL        i
  -------         ENDDO         
  C:0B32H         LINE#         981
  C:0B32H         LINE#         982
  C:0B32H         LINE#         984
BL51 BANKED LINKER/LOCATER V5.00                                                      05/05/2011  10:38:39  PAGE 23


  C:0B34H         LINE#         985
  C:0B36H         LINE#         986
  C:0B38H         LINE#         987
  C:0B38H         LINE#         988
  C:0B43H         LINE#         989
  C:0B47H         LINE#         990
  -------         ENDPROC       READ24C02
  -------         PROC          TEST
  -------         DO            
  D:0004H         SYMBOL        m
  D:0003H         SYMBOL        t
  -------         ENDDO         
  C:09DEH         LINE#         995
  C:09DEH         LINE#         996
  C:09E0H         LINE#         997
  C:09E3H         LINE#         998
  C:09E3H         LINE#         999
  C:09E6H         LINE#         1000
  C:09E9H         LINE#         1001
  C:09F0H         LINE#         1002
  C:09F0H         LINE#         1003
  C:09F2H         LINE#         1004
  C:09FAH         LINE#         1005
  C:09FCH         LINE#         1006
  -------         ENDPROC       TEST
  -------         PROC          MAIN
  -------         DO            
  D:0005H         SYMBOL        m
  -------         ENDDO         
  C:048BH         LINE#         1014
  C:048BH         LINE#         1015
  C:048BH         LINE#         1018
  C:048EH         LINE#         1019
  C:0491H         LINE#         1021
  C:0494H         LINE#         1023
  C:049DH         LINE#         1024
  C:04A3H         LINE#         1026
  C:04A3H         LINE#         1027
  C:04A3H         LINE#         1028
  C:04A6H         LINE#         1029
  C:04A9H         LINE#         1030
  C:04A9H         LINE#         1031
  C:04ACH         LINE#         1033
  C:04ACH         LINE#         1034
  C:04AFH         LINE#         1035
  C:04B2H         LINE#         1036
  C:04B2H         LINE#         1037
  C:04B5H         LINE#         1038
  C:04B5H         LINE#         1040
  C:04B8H         LINE#         1041
  C:04BAH         LINE#         1042
  C:04C5H         LINE#         1044
  C:04C8H         LINE#         1046
  C:04C8H         LINE#         1047
  C:04CBH         LINE#         1048
  C:04CEH         LINE#         1049
  C:04D1H         LINE#         1050
BL51 BANKED LINKER/LOCATER V5.00                                                      05/05/2011  10:38:39  PAGE 24


  C:04D4H         LINE#         1051
  C:04D7H         LINE#         1052
  C:04D7H         LINE#         1053
  C:04DAH         LINE#         1054
  C:04DDH         LINE#         1055
  C:04DFH         LINE#         1056
  C:04DFH         LINE#         1058
  C:04E2H         LINE#         1059
  C:04E2H         LINE#         1060
  C:04E5H         LINE#         1061
  C:04E8H         LINE#         1062
  C:04EBH         LINE#         1064
  C:04EEH         LINE#         1065
  C:04F1H         LINE#         1066
  C:04F4H         LINE#         1067
  C:04F4H         LINE#         1068
  C:04F4H         LINE#         1069
  C:04F7H         LINE#         1071
  -------         ENDPROC       MAIN
  -------         PROC          _DISP_TEMP_ALARM
  D:0007H         SYMBOL        addr
  D:0005H         SYMBOL        num
  C:064BH         LINE#         1079
  C:064BH         LINE#         1080
  C:064BH         LINE#         1081
  C:0659H         LINE#         1082
  C:0661H         LINE#         1083
  C:066BH         LINE#         1084
  C:0677H         LINE#         1086
  C:067CH         LINE#         1087
  C:067CH         LINE#         1088
  C:067FH         LINE#         1089
  C:0684H         LINE#         1090
  C:0687H         LINE#         1091
  C:0687H         LINE#         1093
  C:068AH         LINE#         1094
  C:068FH         LINE#         1095
  C:0694H         LINE#         1096
  -------         ENDPROC       _DISP_TEMP_ALARM
  -------         PROC          TIME0
  C:0AB4H         LINE#         1102
  C:0AB8H         LINE#         1104
  C:0ABBH         LINE#         1105
  C:0ABEH         LINE#         1106
  C:0AC0H         LINE#         1107
  C:0AC7H         LINE#         1108
  C:0AC7H         LINE#         1109
  C:0ACAH         LINE#         1110
  C:0ACCH         LINE#         1111
  C:0ACCH         LINE#         1112
  -------         ENDPROC       TIME0
  -------         PROC          _SPK
  D:0006H         SYMBOL        addr
  C:0B1BH         LINE#         1119
  C:0B1DH         LINE#         1120
  C:0B1DH         LINE#         1121
  C:0B20H         LINE#         1122
BL51 BANKED LINKER/LOCATER V5.00                                                      05/05/2011  10:38:39  PAGE 25


  C:0B20H         LINE#         1123
  C:0B23H         LINE#         1124
  C:0B25H         LINE#         1125
  C:0B27H         LINE#         1127
  C:0B27H         LINE#         1128
  C:0B2CH         LINE#         1129
  C:0B31H         LINE#         1130
  C:0B31H         LINE#         1131
  -------         ENDPROC       _SPK
  -------         PROC          TEMP_COMPARE
  C:0699H         LINE#         1136
  C:0699H         LINE#         1137
  C:0699H         LINE#         1138
  C:06A0H         LINE#         1139
  C:06A0H         LINE#         1140
  C:06A2H         LINE#         1141
  C:06A4H         LINE#         1142
  C:06A6H         LINE#         1144
  C:06ADH         LINE#         1145
  C:06ADH         LINE#         1146
  C:06AFH         LINE#         1147
  C:06B1H         LINE#         1148
  C:06B3H         LINE#         1150
  C:06B6H         LINE#         1151
  C:06B6H         LINE#         1152
  C:06BBH         LINE#         1153
  C:06BEH         LINE#         1154
  C:06C1H         LINE#         1155
  C:06C3H         LINE#         1157
  C:06C3H         LINE#         1158
  C:06C8H         LINE#         1159
  C:06CDH         LINE#         1160
  C:06CDH         LINE#         1161
  C:06D0H         LINE#         1162
  C:06D0H         LINE#         1163
  C:06D5H         LINE#         1164
  C:06D8H         LINE#         1165
  C:06DBH         LINE#         1166
  C:06DBH         LINE#         1168
  C:06DBH         LINE#         1169
  C:06E0H         LINE#         1170
  C:06E5H         LINE#         1171
  C:06E5H         LINE#         1172
  -------         ENDPROC       TEMP_COMPARE
  -------         PROC          _SET_TEMPALARM_FLASH
  D:0004H         SYMBOL        addr
  D:0005H         SYMBOL        num
  C:0A3CH         LINE#         1177
  C:0A3EH         LINE#         1178
  C:0A3EH         LINE#         1179
  C:0A41H         LINE#         1180
  C:0A41H         LINE#         1181
  C:0A47H         LINE#         1182
  C:0A4AH         LINE#         1183
  C:0A4AH         LINE#         1185
  C:0A4AH         LINE#         1186
  C:0A4FH         LINE#         1187
BL51 BANKED LINKER/LOCATER V5.00                                                      05/05/2011  10:38:39  PAGE 26


  C:0A54H         LINE#         1188
  C:0A57H         LINE#         1189
  C:0A5AH         LINE#         1190
  C:0A5AH         LINE#         1191
  -------         ENDPROC       _SET_TEMPALARM_FLASH
  -------         PROC          _KEY_SET
  D:0004H         SYMBOL        num
  C:0916H         LINE#         1196
  C:0918H         LINE#         1197
  C:0918H         LINE#         1198
  C:091BH         LINE#         1199
  C:091BH         LINE#         1200
  C:091EH         LINE#         1201
  C:0923H         LINE#         1202
  C:0927H         LINE#         1204
  C:092AH         LINE#         1205
  C:092AH         LINE#         1206
  C:092DH         LINE#         1207
  C:092DH         LINE#         1208
  C:0930H         LINE#         1209
  C:0934H         LINE#         1210
  C:0937H         LINE#         1211
  C:0939H         LINE#         1212
  C:0939H         LINE#         1213
  -------         ENDPROC       _KEY_SET
  -------         PROC          SET_TEMP_ALARM
  C:04F9H         LINE#         1218
  C:04F9H         LINE#         1219
  C:04F9H         LINE#         1220
  C:04FCH         LINE#         1221
  C:04FFH         LINE#         1222
  C:04FFH         LINE#         1223
  C:0502H         LINE#         1224
  C:0504H         LINE#         1225
  C:0507H         LINE#         1226
  C:0507H         LINE#         1228
  C:050AH         LINE#         1229
  C:050AH         LINE#         1230
  C:050FH         LINE#         1231
  C:0516H         LINE#         1233
  C:0519H         LINE#         1234
  C:0519H         LINE#         1235
  C:051CH         LINE#         1236
  C:051EH         LINE#         1237
  C:0520H         LINE#         1238
  C:0522H         LINE#         1239
  C:0529H         LINE#         1240
  C:052CH         LINE#         1241
  C:052CH         LINE#         1242
  C:052EH         LINE#         1243
  C:0531H         LINE#         1244
  C:0531H         LINE#         1245
  C:0536H         LINE#         1246
  C:053DH         LINE#         1248
  C:0540H         LINE#         1249
  C:0540H         LINE#         1250
  C:0543H         LINE#         1251
BL51 BANKED LINKER/LOCATER V5.00                                                      05/05/2011  10:38:39  PAGE 27


  C:0545H         LINE#         1252
  C:0547H         LINE#         1253
  C:054EH         LINE#         1254
  C:0551H         LINE#         1255
  C:0554H         LINE#         1256
  C:0554H         LINE#         1257
  C:0556H         LINE#         1258
  -------         ENDPROC       SET_TEMP_ALARM
  -------         ENDMOD        SOFTWARE

*** WARNING L13: RECURSIVE CALL TO SEGMENT
    SEGMENT: ?PR?KEYDOWN?SOFTWARE
    CALLER:  ?PR?ECODECHANGE?SOFTWARE

*** WARNING L16: UNCALLED SEGMENT, IGNORED FOR OVERLAY PROCESS
    SEGMENT: ?PR?CODEDISPLAY?SOFTWARE

*** WARNING L16: UNCALLED SEGMENT, IGNORED FOR OVERLAY PROCESS
    SEGMENT: ?PR?TEST?SOFTWARE

Program Size: data=56.1 xdata=0 code=3018
LINK/LOCATE RUN COMPLETE.  3 WARNING(S),  0 ERROR(S)
